:030000000219FDE5
:03000B000200A848
:03002B000201636C
:03005B000202EDB1
:030073000202D3B3
:1000800002030406080C10182030406080040608A3
:100090000C10182030406080A0C000070F1F3F05E3
:1000A000050D050305030302C2AFC0D0C0E0206206
:1000B00017E5256002E473E525F4F58A758B00D217
:1000C00062D0E0D0D0D2AF3285268AC262E526F473
:1000D0006035306803207210758B00D0E0D0D0D22C
:1000E00092D291D290D2AF32D292D291D290206E4F
:1000F0000C206609740AD5E0FDE57E4290758B0000
:10010000D0E0D0D0D2AF32758A00C28DD26201FD6C
:1001100001B7306805206602C29201B73068052039
:100120006602C29101B7306805206602C29001B72D
:10013000C29330680A2066077408D5E0FDC29201B8
:10014000B7C29430680A2066077408D5E0FDC291F2
:1001500001B7C29530680A2066077408D5E0FDC271
:100160009001B7C2AFC2AD53E6EFC0D0C0E0D2D36A
:10017000D2AFC2CEE52A6007207449152A21C4787F
:1001800000790020742EE580307E01F430E402789E
:10019000FF53DACF207E0343DA20307E0343DA10A8
:1001A000C2D8C271E580307E01F430E40279FFC329
:1001B000E89970CB306103752A18207403752A18EA
:1001C000885FD27020740DE52B6004152B21D44379
:1001D000DA01C2D82070024136A85F206102C270E5
:1001E000207431C3E894F0400374F0F8E8C4540F6D
:1001F00028F87984B703024114C313C3138721205D
:100200000802C313200A06C3C898F8411428F850FE
:100210000374FFF8C3E895685003E568F88822E5A1
:100220002D54066011E533C313C31324062522F5AC
:100230002250037522FF852224A824C3E524956457
:100240004002A8648825E5697002417AC3E8AA697A
:100250009A5003E8FAE4F9EAC333FBE56BF45B294F
:10026000400D256AF8E56A6002156A400B417A0A7A
:10027000C3E56A9A5002056A78FF8826C26EC3E514
:100280002694F84002D26EC3E52594404002D26421
:1002900020CF0AD0E0D0D043E610D2AD32C2CF0595
:1002A0003A7801E52A6005307402152AC3E55F94A7
:1002B00001400575620041C9756300756C00E56217
:1002C0002401F56250037562FFD0E0D0D043E61000
:1002D000D2AD32C2AFC0D053E67FC2607591008507
:1002E0005694855795759104D0D0D2AF32C2AF5392
:1002F000E6EFC2ADC0D0C0E0C0F0D2D3D2AFA8FB11
:10030000A9FCC2D8307102615453DACF207E034376
:10031000DA10307E0343DA20D271E580307E01F4BA
:1003200020E402612B88278928A18153DACF207E1F
:100330000343DA20307E0343DA10C2D8C27130742E
:1003400002A16D7800E580307E01F430E402A16DF9
:10035000885FA15553DACF207E0343DA20307E0335
:1003600043DA10C271206102812D53DACF207E035F
:1003700043DA10307E0343DA20C2D8D271885A891A
:100380005BC3E89558F8E99559F97B007E087A0037
:10039000C3E8948CE994005005755E00811F8821A4
:1003A00078A2E6A8216055C3E894C8E994005008F3
:1003B000E4D2E4FB7A0A61FAC3E89468E994015054
:1003C00008E4D2E3FB7A0F61FAC3E894D0E994021F
:1003D0005008E4D2E2FB7A1E61FAC3E894A0E994E3
:1003E000055008E4D2E1FB7A3C61FAC3E89498E94D
:1003F00094085008E4D2E0FB7A787E00C3E8955C6C
:10040000FCE9955DFD30E70AECF42401FCEDF434E1
:1004100000FD755E00C3EC9AED9E5003755E018889
:100420005C895D855A58855B597802A155C3E8956A
:1004300027F8E99528F9307C02A139307B02A139EF
:10044000307A02A1322075028150E9FDE8FC816F0B
:10045000E9C313F9E813F8307902A132E9C313F9BB
:10046000E813F8307802A132E9C313FDE813FC2049
:0E047000612CC3EC941CED940240028186EDD9
:10047E00701EC3EC94C850180529E5297002152981
:10048E00C3E529940A5002A16D755F00D270A16D6B
:10049E00E529600215297888E6F97400207F08782E
:1004AE0096B90302789EE624FAFEE43400FFC3EC0C
:1004BE009EFCED9FFD9208B90310A208500720760E
:1004CE0009D27681D8307602C276A2085016B903C8
:1004DE000DECF42401FCEDF43400FD0204F278007E
:1004EE007900A139B90315EC33FCED33FDC3EC945F
:1004FE000AFCED9400FD50047C007D00C3EC94FFDB
:10050E00ED9400400678FF7900A139EC8575F0A4D2
:10051E00C5F0A2F733F87900400302055578FF794C
:10052E0000020555E9C313F9E813F8307C0EE960B3
:10053E000278FFC3E81338F8E43400F9C3E894FFF7
:10054E00E99400400278FF885FD270206102A16DAD
:10055E00741FF4552F4BF52FC274EB7002D27475C5
:10056E002A18307403752A0A306102A1812074039F
:10057E0053DAFE207403752B06D0F0D0E0D0D0D223
:10058E00AD43E6103279010205B179030205B17966
:10059E000A0205B1791E0205B179640205B179C866
:1005AE000205B17817E4D5E0FDD8FAD9F6227A140F
:1005BE007B780205D87A107B8C0205D87A0D7BB435
:1005CE000205D87A0B7BC80205D87902B27DE4C247
:1005DE0094D5E0FDC291D5E0FDD291D5E0FDD29447
:1005EE00D5E0FDC292E576D5E0FDD2927496D5E0C7
:1005FE00FDD9D9EAF8D5E0FDD8FBDBCEC29422C3F3
:10060E007C007D0075F00005F0EA33FAEB33FB5009
:10061E00F6EB13FBEA13FAC3E9FFE8FEE89AF8E9F2
:10062E009BF95004EFF9EEF8B3EC33FCED33FDD546
:10063E00F0DFEDF9ECF822E889F08A20D2D4F8A99F
:10064E00F07B0030F70B7BFFF42401F8E9F4340063
:10065E00F9E88520F0A4ADF0F8E98520F0A4AFF01C
:10066E00FEED2EF974003FFA7C04C3EA13FAE91387
:10067E00F9E813F8DCF48BF030F70AE8F42401F80B
:10068E00E9F43400F9E889F0C2D4F8A9F02222C3C3
:10069E00E54113F9E54013F8C3E54598F8E54699A9
:1006AE00F9500CC3E89480E994FF40160206D4C3B7
:1006BE00E8947FE9940050030206D4787F79000213
:1006CE0006D4788079FF884A894B22E54A2547F877
:1006DE00E54B3548F9854B20E4300701F43549FAEE
:1006EE0030E709C3EA94F04015020712C3EA940FEB
:1006FE00500302071278FF79FF7A0F020712780073
:10070E0079007AF0C3E5249564500AC374019524E8
:10071E00500B020730E54B20E70E020730E54B3059
:10072E00E706884789488A492278A4E6FAC3E54A4B
:10073E0033F8E54B33F9D145E930E70BC3E8948044
:10074E00E994FF4013E16AC3E8947FE994005002F4
:10075E00E16A787F7900E16A788079FFE820E71511
:10076E00C3E52398F84009C3E894014003020791BA
:10077E007801020791E8F424012523F840030207CB
:10078E009178FF884C2278A5E6FAA848A949D14568
:10079E00E930E70CC3E89401E994FF40160207C55F
:1007AE00C3E894FFE9940050030207C578FF79006F
:1007BE000207C5780179FFE920E715C3E54C98F8E3
:1007CE004009C3E8940140030207EC78010207ECEC
:1007DE00E8F42401254CF840030207EC78FF882446
:1007EE002278FFC26420693D206A12D264C3E541BB
:1007FE00940A4009C3E52594405002C26479A1E7EA
:10080E006023E541601F74FF8541F0848539F03027
:10081E006A0375F005A4F8C5F0600278FFC3E89589
:10082E00675002A867886622C3E5409440E541946C
:10083E0001E5665003140147046002F566220208C2
:10084E004F2275E890227883E6FFE5E820ECF7A8C2
:10085E00BDA9BE0573C3E57394084052757300E9D4
:0D086E00FA79A0E76044EA7007E574601BAA
:10087B0002088AC3E895746010E5745006600C1486
:10088B000208960460F9020896E574F574C394584F
:10089B00401B7564C0C394044013756480C39404F7
:1008AB00400B756440C39404400375640075BB032F
:1008BB0022E564F460020564E573B4070375BB10AD
:1008CB0022743279A687F0A4C5F0A2F733F8C3E8F7
:1008DB0095644002A8648822882488258826886726
:1008EB00227540007541F022C2AF75C820A8CCA973
:1008FB00CDAA3A30CF010A75C824D2AFAB3BAC3C82
:10090B00883B893CC3E89BF8E99C206908F9306770
:10091B000241082165AD3D8A3DF9EA9DFA600478F4
:10092B00FF79FFAE3EAF3F8B3E8C3FC3EC9FFCC3CA
:10093B00E99CF542A83BA93CC3E89EF8E99FF9C3A3
:10094B00E54113FBE54013FAE82AF540E93BF54195
:10095B0050067540FF7541FF21AFAA40AB41AC403B
:10096B00AD417E047F02C3EB940440021E1FC3EB18
:10097B00940840021E1FC3ED13FDEC13FCDEF7C3FE
:10098B00EA9CFAEB9DFBEF6009C3E913F9E813F856
:10099B00DFF7EA28FAEB39FB8A408B4150067BFFE5
:1009AB008B408B41C3EB94025002D2673069047FBA
:1009BB000321DA7892E6FFC3E537948240110FC327
:1009CB00E53794A040010FC3EF940640027F057EEC
:1009DB0005E541C4540FF9E541C454F0F8E540C4B2
:1009EB00540F28F8C3E89EFAE99400FB4009C3EAC8
:1009FB009402EB940050047A02E4FB4154AA40ABFE
:100A0B0041EBC4FEEAC4540F4EFCC3EA9CFAEB94D0
:100A1B0000FBC3E813C313F8EA28FAEB3400FB8A94
:100A2B00408B41C3EB94024002C2677805EBC4FED6
:100A3B007B00EAC4540F4EFAC3EA98FA4005C394FC
:100A4B000250027A027892E6FF30600241548552DE
:100A5B0056855357D26043E680C3E49AF8E49BF97A
:100A6B0030670241EEE8FAE9FBD3E913FDE813FC2A
:100A7B0088528953C3EF94036038EF20E00DE82CC4
:100A8B00F8E93DF9ECFAEDFB020AA9E828F8E93997
:100A9B00F9C3E82402F8E93400F97AFE7BFFC3EFCF
:100AAB009403400E8A548B55884E894F8C508D5130
:100ABB006122885489558A4E8B4F8C508D513069E9
:100ACB0020C3E53394034019E542A2E713F8E5553B
:100ADB00F4240138400B20E7087554FFF42401F58A
:100AEB00556122E8FAD3E813FC8852C3EF940360F4
:100AFB0020EF20E007E82CF8ECFA610EE82824023E
:100B0B00F87AFEC3EF940340088A54884E8C5061E8
:100B1B002288548A4E8C50E56BC3335002646BF5BC
:100B2B006B306002612C753402D26043E680E52D98
:100B3B0054066026A840A941C3E913F9E813F8C28B
:100B4B00AF53E67F759100C3E498F594E499F5955E
:100B5B00759104D26043E680D2AF22D26575440012
:100B6B00752000306B03752040020B85D2657544F0
:100B7B0000752040306B03752000D2AF78012067E1
:100B8B0022E52D54066002C265C3E541940540136E
:100B9B007802940540087803940540027806306982
:100BAB0002780A206019E544601530690AC3E53301
:100BBB0094034003D53406D2AFD26C81577134D233
:100BCB00AF0000C2AF206726E541C3FB940F400284
:100BDB007B0FEB240530730123306A0274282062EB
:100BEB000123F93069027982E58BC39940B505443D
:100BFB00E59BF45440B52002814130690A08C3E8F3
:100C0B00940A40010861AE2065026185C26553E616
:100C1B007F7591003067107594007595FE75910482
:100C2B00D26043E6806185AE40AF41C3E49EF5944C
:100C3B00E49FF5958128C3E533940250026185301A
:100C4B0065026185D802815561AEC26C53E67F7532
:100C5B009100855494855595759104854E56854F15
:0E0C6B0057D26043E680D2AFE52D54066008F4
:100C7900206A020533020C91306C0D206B0A206545
:100C89000715811581021520227800306405306529
:100C9900027801E53775F007A4F9E5F028F5F0E9E0
:100CA900A2F013A2F113A2F213F537C394785003FB
:100CB900753778C3E53795384008D266D292D29114
:100CC900D29030600281CB855056855157D260430E
:100CD900E68022D2A0207D11C2AF754302C294D210
:100CE90093D2AF759F10020EB7C2AF754302C2947B
:100CF900D295D2AF759F10020EB7C2A030724320B1
:100D09007D20C2AF754303900141757E10D290C218
:100D190095306204C291A123D294D2AF759F20026B
:100D29000EB7C2AF754303900141757E10D292C2CE
:100D390093306204C291A143D294D2AF759F00024D
:100D49000EB7207D17C2AF75430390011CD29030B6
:100D59006202C291D2AF759F20020EB7C2AF75432E
:100D69000390011CD292306202C291D2AF759F00EA
:100D7900020EB7D2A0207D11C2AF754304C293D22F
:100D890095D2AF759F00020EB7C2AF754304C295E5
:100D9900D293D2AF759F20020EB7C2A03072432002
:100DA9007D20C2AF754305900130757E08D291C28E
:100DB90094306204C292A1C3D293D2AF759F10023C
:100DC9000EB7C2AF754305900152757E20D291C20C
:100DD90094306204C290A1E3D295D2AF759F1002FC
:100DE9000EB7207D17C2AF754305900112D291301D
:100DF9006202C292D2AF759F10020EB7C2AF75439D
:100E090005900126D2913062EBC290D2AF759F1046
:100E1900020EB7D2A0207D11C2AF754306C295D28A
:100E290094D2AF759F20020EB7C2AF754306C29325
:100E3900D294D2AF759F00020EB7C2A03072422081
:100E49007D20C2AF754301900152757E20D292C2B6
:100E590093306204C290C163D295D2AF759F0002EC
:100E69000EB7C2AF754301900130757E08D290C2AA
:100E790095306204C292C183D293D2AF759F20C1CB
:100E8900B7207D16C2AF754301900126D292306218
:100E990002C290D2AF759F00C1B7C2AF754301902E
:100EA9000112D290306202C292D2AF759F20C266FF
:100EB90022900110757E00D292D291D290C293C233
:100EC90094C295C26222788076FF0876FF0876FF81
:100ED9000876FF08760308760408760A0876030878
:100EE9007601087601788C76010876FF0876FF0886
:100EF90076FF0876FF0876FF0876030876FF0876FE
:100F0900FF0876FF0876250876D00876FA0876FA7B
:100F19000876040876FF08760108760008767A08CC
:100F290076FF0876010876010876000876032278AC
:100F390087E6FFC272BF0302D2727888E6C39403C0
:100F49006008C27DE630E102D27DC27E7889E63052
:100F5900E102D27EC3EF94026008758E01D273025A
:100F69000F70758E00C273227880E614900080930A
:100F790078A4F67881E6149000809378A5F67886AF
:100F8900E61490008D9378A6F6789CE67538FF757F
:100F9900390CB402067538A075390AB403067538D8
:100FA9008275390578A3E61490009A93F569D1BA48
:100FB90022227896E6FA7897E6FB7888E6B4030564
:100FC900C3EB940EFB307F047A007BFFC3EB9AFCE2
:100FD900C3948250027C827575000575EC8575F0A5
:100FE900A4C3E5F0947D40F222D27FF1BB1205A2A1
:100FF9007A007B007C10120598E55F2AFA74003BA1
:10100900FBDCF37C04C3EB13FBEA13FADCF7FEC247
:101019007F120FBB22E5EF20E60375200005209023
:101029003FFFE520146006901DFF146000930460E3
:101039000375EF1253D9BF7581C043FF8012059321
:1010490075EF0243B203E5B3240420E70DF521E56A
:10105900E320E0068521B343E301120EBA7580FF50
:0F10690075A40075F1D475D4EF75908775A54007
:1010780075F2FF75D5BF75A60175E24275DB467539
:10108800EA02E4F8F6D8FD756B01120ECF1215626C
:1010980078988676753001C2AF1205AC1205BC127D
:1010A80005A21205C31205A21205CA1205A212163C
:1010B8007B1205AC1205AC1205A7C2AF78FA79FA13
:1010C800308407D9FBD8F7021C00120F38120F71B1
:1010D800120FBA120FBB78988676120EBA7588501E
:1010E80075891275C82475910475D84075A822753C
:1010F800B80275E690759B80759D0075D10E75BC1C
:101108005875BB0375BA1175E880120593D2AF12F2
:10111800084C53DACF207E0343DA20307E0343DACB
:101128001043DA01C2D8C2711205ACD2617B037ACE
:101138000CE55E70077A0CDB030210C21205A220D0
:1011480070030210C2C270E55FC3940240E1E52F4C
:10115800541F856160F561B560D5DAD5C26153DA8F
:10116800CF207E0343DA20307E0343DA10C2D8C290
:101178007178A2E67008D274E52F54E0F52FC27595
:101188007529001205A7307409C3E529940A40029D
:10119800D27512059878023074027800C3E55F981A
:1011A80040F0C2AF1205BC1205BC1205BCD2AF128A
:1011B80005AC754D007888E6B4030241A212059883
:1011C800788CE6C3940150030212A2E530C394015F
:1011D80050030212A2207435C3E55F94FF50030246
:1011E80012A2C2AF1205D1D2AF1205A7C3E55F9410
:1011F8000150EFC2AF1205BC12059D1205BCD2AF5B
:101208001205A7C3E55F94FF40E90217007F05D2E6
:101218007F120FBB1205A7C2AFC27F120FBBAE5F12
:10122800C3E55F947FD2AF407B120593C2AF12052E
:10123800D1D2AFDFDA120FF2C3EE94057897F61227
:1012480005AC1215A41216837F0AD27F120FBB12A7
:1012580005A7C2AFC27F120FBBAE5FC3E55F947F25
:10126800D2AF50E4120593C2AF1205BC12059D120D
:1012780005BCD2AFDFD4120FF2EE24057896F61231
:1012880005AC1215A41216B21205A7120FBBC3E5BE
:101298005F94FF500221DD021700C3E55F954D40C2
:1012A80003855F4D1205A778017988E7B4030278B2
:1012B80005C3E55F98400221BDC2AF1205D11205F2
:1012C800D11205D1D2AF1205AC753000E4F531F575
:1012D800320531E531F470390532789AE678191417
:1012E8006012783214600D787D14600878FA146002
:1012F80003753200C3E53298401715327531B4785A
:10130800998676C2AF1205D1D2AF78988676120543
:10131800A712059DE52A700530740201C2780120E4
:1013280074027806C3E55F9840A77888E6C39403FB
:1013380060031205A7E52A70030210C2C2AF120E9D
:10134800BAE4F522F523F524F525F526F56AD2AF9A
:101358007885E6C333F568E4F545F546F547F5487D
:10136800F549F573F52CF52DF53775730875BB1030
:10137800120593120850E5E820ECFBA8BDA9BEE9C8
:101388007001F8887412085475730875BB10788753
:10139800E6FE7602120F387887EEF6C2AF7564FF64
:1013A8001208CC852264852265852266D2AF752213
:1013B8000175240175250175260185636C756D011C
:1013C8007888E6B40307C27D307602D27DD268D22F
:1013D80069753300120E1C120E431208EC1208F342
:1013E8001208EC1208F31208EC021401C2AF120F33
:1013F80038D2AF75730075BB03120B7712069C12B7
:101408000C92120CDC1208F3120B66306D031206F4
:101418009D2067031207EF306703120836120C92FB
:10142800120D031208F3120B77306D031206D9124E
:101438000C92120D7C1208F3120B66306D03120722
:1014480037120C92120DA31208F3120B77306D03AA
:10145800120794120C92120E1C1208F31208501262
:0E1468000B66120C92120E431208541208F377
:10147600306932206B2F85676485676585636C7577
:101486006D0179187A0CC3E53399400CC269D26AAA
:101496008A357564FF0214ABC3E55F94014003020D
:1014A6001401021528306A1B206B18E535147004E8
:1014B600C26A61F4F535C3E55F9401400302140185
:1014C600021528753600C3E5627882985054307448
:1014D60004E52A604D7888E6B40317207D0520765A
:1014E6000781F830760281F8206B07D26B85676436
:1014F600814078F0306B058567647820C3E54198B4
:1015060050028101306B1BC26BC27D307602D27DE8
:10151600D26A75351285676481010536E55F60021A
:10152600A12B753600C2AF120EBA7887E6FE760298
:10153600120F387887EEF6E4F522F523F524F52523
:10154600F526F568C268D2AF120593120EBA30744A
:1015560009C3E5369405400201C241D4901A0D78BC
:10156600201215E6E520B45A0CA31215E6E520B4C0
:10157600A503021584120ECF1215A40215A3901A04
:101586000378807B0A1215E6A308DBF9901A0F7818
:101596008C7B181215E6A308DBF9901A2722C2AF36
:1015A6001216251215FF901A00740E1215EBA3746D
:1015B600041215EBA374141215EB901A0378807BB2
:1015C6000A1215EAA308DBF9901A0F788C7B181219
:1015D60015EAA308DBF9121638121616901A2722F6
:1015E600E493F622E6438F01538FFD75EF0275B73C
:1015F600A575B7F1F0538FFE22438F02438F017515
:10160600EF0275B7A575B7F1901A0DF0538FFC224E
:10161600901A0D745AB1EB901A0E74A5B1EB227A9A
:101626003079D07820901A40B1E6E520F709A3DAA0
:10163600F7227A3079D0901A40E7B1EB09A3DAF9AC
:1016460022AB77A878BB01027984BB02027985BBFD
:1016560003027986BB04027992BB05027987BB0631
:101666000279A3BB0702799CBB08027988BB0902F1
:101676007989E8F7227C051205ACDCFB22C2AF12A1
:1016860005BC1205C31205CA1205D112059D120525
:10169600BC1205C31205CA1205D112059D1205BC5E
:1016A6001205C31205CA1205D1D2AF22C2AF120566
:1016B600D11205CA1205C31205BC12059D1205D129
:1016C6001205CA1205C31205BC12059D1205D112D8
:1016D60005CA1205C31205BCD2AF22AE77AF78C2D7
:1016E600AF1205BC1205BC1205BC12059DDEF21236
:1016F60005D112059DDFF8D2AF22D183D17BD17BF4
:10170600757701757801757900D1E17C05AD5F12B9
:1017160005ACC3ED955F70F5C3E55F9401400AC360
:10172600E55F94FF403202173CD147B1A4D183C292
:10173600AF75EF12D17BDCD50579C3E579940350FB
:101746000280C6D17B0578E5771490009F93F80850
:10175600C3E57898500280AED17BD17B0577C3E58F
:1017660077940A5002809C120ECFB1A4C2AF75EFD7
:0317760012D17B12
:0319FD0002101EB7
:101A00000E0414FFFFFFFF03040A0301015AA5019E
:101A1000FFFFFFFFFF03FFFFFF25D0FAFA04FF01DE
:081A2000007AFF01010003FF41
:101A400023484B696E67323041232020202020201C
:101A500023424C48454C4923463333302320202031
:101A60002020202020202020202020202020202076
:101C0000C2AFC2D353D9BF7581C043B20343FF8073
:101C1000752438752503B1C975EF0275E24043F1AB
:101C20001053A4EF75D400D2847DFA780379E67C52
:101C300010752200752300901DD67B0675249875BB
:101C400025013084028142208408D8FBD9F9DCF7D1
:101C500081B4308408D8FBD9F9DCF781B4B189E4C8
:101C600093A3C39A6004DDC381B4DBDBB17B600264
:101C7000812B7B08E493FAA3B15CDBF87A30B15C8A
:101C8000752200752300B17BEAFCEBFDC3ED94FEE9
:101C9000400EB17B8A278B28ED30E0048A828B834B
:101CA000B17B7AC270D8C3ED94FE601350CEBD00F4
:101CB00025EC60097520007521FF0200008100A855
:101CC00027A9280809D804D90281D3B17FEA89AAB3
:101CD000F281C50D81A0C3ED94035049EDA2E092BD
:101CE000007AC5C3E5829400E583941C50902000DF
:101CF00010438F02438F0175B7A575B7F1F030001F
:101D00001FA827A9280809438F01538FFDD804D99C
:101D100002A12089AAE275B7A575B7F1F0A3A10DBC
:101D2000538FFC817C7AC1BD030CE493A3FAB140CC
:101D3000DCF8B138817C817EAA22AB23B15CEBFA5E
:101D4000EA6222752608C3E52313F523E52213F57D
:101D50002250066323A0632201D526EAB1C9B1C986
:101D600075260AEAF4200102D284300102C284B14D
:101D7000C9C3134002C201D526EB22B17FEAFB2082
:101D80008402A17F308402A184752608AE24AF2589
:101D9000C3EF13FFEE13FEB1CDB1C9C3EA13308414
:101DA000024480FA30E703632201C3E52313F523DD
:101DB000E52213F52250066323A0632201D526D91C
:101DC000E52265236523F52222AE24AF250E0FDE22
:101DD000FEDFFCD20122424C48656C693437316326
:041DE000F3300601D5
:00000001FF
